:100EAA0000C000F900A400B000990092008200F886
:100EBA00008000900088008300C600A10086008E92
:070F7500C41313135401FF24
:0A0F7C00E51125E0F511EF42112206
:0D10BA00E51125E0F511EFF454014211227B
:0411AB00EF521122CC
:07116E00EFF45401521122BD
:0411AF00EF421122D8
:07117500EFF45401421122C6
:0E108200E511F45401FFE51154FE4FF5112263
:0610FB005401FF120F7CFE
:06110100E5115401FF227C
:0D10C700E511C313FFE51154015FF511227F
:0D10D400E511C313FFE51154014FF5112282
:0E109000E51125E0F511EDF45F540142112247
:0E109E00E51125E0F511EFF45D540142112239
:08000300EDF45F5401521122DB
:08115600EFF45D540152112277
:08115E00EDF45F54014211227F
:08116600EFF45D540142112277
:07117C00EDF45F5401FF22B6
:07118300EFF45D5401FF22AF
:0D10E100E51825E0FFE51154014FF5182238
:0D10EE00E5185401FFE51154FE4FF51122E5
:100F6200E5185401FFE51154FE4FF511E518C313BE
:030F7200F518224D
:101063008E5D8F5EE55E2DFFE55D3C8FF0020ACF5E
:100F86008E5F8F60C3E5609DFFE55F9C8FF0020A70
:010F9600CF8B
:09114D00120A0EEE8FF0020ACF27
:0F1073008B5A8A5B895C120A20EE8FF0020ACF3B
:07118A00E475F001020A9771
:0711910074FFF5F0020A975C
:100F97008E618F62E5615CFFE5625DCF8FF0020ACB
:010FA700CF7A
:100FA8008E638F64E5634CFFE5644DCF8FF0020AD2
:010FB800CF69
:100FB9008E658F66E5656CFFE5666DCF8FF0020A79
:010FC900CF58
:100FCA00EFF4FFEEF4FEEF2401FFE43E8FF0020A95
:010FDA00CF47
:06119F00EFF45401FF22F1
:0611A500EE8FF0020ACFFC
:0A114300EFF4FFEEF48FF0020ACF84
:100E54008B4B8A4C894D120A6CFFAEF0AB4EAA4FF5
:100E6400A950120A6CFDAB4BAA4CA94DE5F08DF0CC
:0F0E7400120ACFAB4EAA4FA950EE8FF0020ACF51
:100B43008E518F528B538A5489557C037DE8120A48
:100B530020EFC454F07B00FAAE51AF527C037DE822
:100B6300120A208C518D52AE51AF527C007D64121B
:100B73000A20EFFEE4EE4202AE51AF527C007D64E8
:100B8300120A208C518D52AE51AF527C007D0A1255
:100B93000A20EFC4F8540FC868FFEEC454F048FEAF
:100BA300EFFBEE4202AE51AF527C007D0A120A20E7
:100BB3008C518D52E5514AFFE5524BAB53AA54A9D0
:070BC30055CF8FF0020ACFAD
:100C49008E568F57E557780CCEA2E713CE13D8F8F6
:100C59007E00540FFF7C037DE8120A0E8E588F59CF
:100C6900E556FF3395E07E00EF540FFF7C007D646D
:100C7900120A0EEF2559F559EE3558F558E557AED4
:100C8900567804CEA2E713CE13D8F87E00540FFF8E
:100C99007C007D0A120A0EEF2559F559EE3558F5F3
:100CA90058E557540F2559F559E43558F5588559DC
:040CB900F0020ACF6C
:100ECA00E51125E0F511C3EF9DEC6480F8EE64802E
:0B0EDA00984004431101225311FE2236
:100EE500E51125E0F511D3EF9DEC6480F8EE648003
:0B0EF500985004431101225311FE220B
:100F0000E51125E0F511D3EF9DEC6480F8EE6480E7
:0B0F1000984004431101225311FE22FF
:100F1B00E51125E0F511C3EF9DEC6480F8EE6480DC
:0B0F2B00985004431101225311FE22D4
:100F3600E51125E0F511EF6D7002EE6C60044311CA
:060F460001225311FE22FE
:100F4C00E51125E0F511EFB50508EEB504044311E4
:060F5C0001225311FE22E8
:100FDB00C3EF9DEC6480F8EE64809850035311FED0
:010FEB0022E3
:100FEC00D3EF9DEC6480F8EE64809840035311FEBF
:010FFC0022D2
:100FFD00D3EF9DEC6480F8EE64809850035311FE9E
:01100D0022C0
:10100E00C3EF9DEC6480F8EE64809840035311FEAC
:01101E0022AF
:0C110700EFB50507EEB504035311FE22FE
:0C111300EF6D7002EE6C60035311FE22C1
:10101F00C3EF9DEC6480F8EE6480984003431101A8
:01102F00229E
:10103000D3EF9DEC6480F8EE648098500343110177
:01104000228D
:10104100D3EF9DEC6480F8EE648098400343110176
:01105100227C
:10105200C3EF9DEC6480F8EE648098500343110165
:01106200226B
:0C111F00EF6D7002EE6C600343110122C2
:0C112B00EFB50507EEB5040343110122E7
:07119800E4FF0FBF0AFC2277
:100E2400E4FEC2B4121198C2B3121198D2B31211D3
:100E340098D2B4121198E4FDEE25E0FE30940343F9
:100E44000601C2B3121198D2B30DBD08EBAF06224E
:10082D000510E510C394054003E4F510E5101460C0
:10083D005B1470030208E914700302093524036088
:10084D00030209877C0090000DE0540FFD25E0FFA9
:10085D00EC33FE74AA2FF582740E3EF583E493FCFF
:10086D00740193FD43040890010AE0FFC4131313B0
:10087D00540130E0057DFF0209DDEF131313541F02
:10088D0020E0030209DD53057F0209DD90000CE035
:10089D00FEA3E07804CEA2E713CE13D8F87C005463
:1008AD000FFD25E0FFEC33FE74AA2FF582740E3E8A
:1008BD00F583E493FC740193FD43040490010BE074
:1008CD0030E0057DFF0209DD90010AE0FFC4540F01
:1008DD0020E0030209DD53057F0209DD90000CE0E5
:1008ED00FF3395E07C00EF540FFD25E0FFEC33FE68
:1008FD0074AA2FF582740E3EF583E493FC74019374
:10090D00FD43040290010BE0FFC31330E0057DFFB2
:10091D000209DD90010AE0FFC413540720E0030231
:10092D0009DD53057F0209DD90000CE0FEA3E078A0
:10093D000CCEA2E713CE13D8F87C00540FFD25E0A2
:10094D00FFEC33FE74AA2FF582740E3EF583E4930B
:10095D00FC740193FD43040190010BE0FF1313544C
:10096D003F30E0047DFF806890010AE0FFC413135F
:10097D00540330E05B53057F805690010BE0F9C4C2
:10098D001313540175F008A4FBAAF0E9C413131353
:10099D00540175F010A4FFE5F04AFAEF4BFBE9C4E2
:1009AD0013540175F004A4FFEA45F0FAEB4FFBE98F
:1009BD00C4540125E0FFE4334AFEEB4FFFE9131366
:1009CD00135401FBEEEF4BF4FFEEF47410FCAD0786
:1009DD007B10C2B3121198EC20E704C2B78002D28B
:1009ED00B7121198ED25E0FDEC33FCD2B31211983E
:1009FD00DBE0D2B7121198C2B5121198D2B502111F
:010A0D009850
:10064700E52E700302082C152E0517E517B40517BC
:10065700AF30EFC4135401F45401FFC43354E0FF27
:10066700E53054DF4FF530E517B40A1CAF30EFC45F
:10067700135401F45401FFC43354E0FFE53054DF51
:100687004FF530051DE4F517E4F568E56813131316
:10069700541F2412F8E6FD7C00E5685407FF740137
:1006A7007E00A807088005C333CE33CED8F9FFEE06
:1006B7005CFEEF5D4E6043E56825E025E0246EF5BE
:1006C70082E43400F583E0FEA3E0FFE56825E0253A
:1006D700E0246CF582E43400F583E0FCA3E0C39FDB
:1006E700EC9E5016E56825E025E0246CF582E4349D
:1006F70000F583E475F001120A56E56825E025E068
:10070700246EF582E43400F583E0FEA3E0FFE5689C
:1007170025E025E0246CF582E43400F583E0FCA3B2
:10072700E0C39FEC9E407AE56825E025E0246CF560
:1007370082E43400FEC3E582946CFFEE9400FE7CF5
:10074700007D02120A207C007D02120A207C007DB7
:1007570008120A20741E2FF8C000E6FFC007E568DC
:1007670025E025E0246CF582E43400FEC3E582949D
:100777006CFFEE9400FE7C007D02120A207C007D57
:1007870002120A207C007D08120A20AF057401A816
:1007970007088002C333D8FCFED0E04ED000F680B5
:1007A70079E56825E025E0246CF582E43400FEC392
:1007B700E582946CFFEE9400FE7C007D02120A2015
:1007C7007C007D02120A207C007D08120A20741E1C
:1007D7002FF8C000E6FFC007E56825E025E0246C98
:1007E700F582E43400FEC3E582946CFFEE9400FECC
:1007F7007C007D02120A207C007D02120A207C0008
:100807007D08120A20AF057401A807088002C333C8
:10081700D8FCF4FED0E05ED000F60568E5686420F9
:06082700600302069222AC
:100D6A00E51DB41E19AF30EFC413135401F4540136
:100D7A00FFC4333354C0FFE53054BF4FF530E51D8F
:100D8A00B43C1CAF30EFC413135401F45401FFC434
:100D9A00333354C0FFE53054BF4FF530E4F51D221C
:03000B00020CBD27
:100CBD00C0E0C0D075D008758CEEAF30EF131313B4
:100CCD005401F45401FF33333354F8FFE53054F736
:100CDD004FF530053AE53A30E0020516E53AB40A2B
:100CED0015AF30EFC45401F45401FFC454F0FFE5C7
:100CFD003054EF4FF530E53AB4141AAF30EFC45419
:100D0D0001F45401FFC454F0FFE53054EF4FF530BA
:0A0D1D00052E753A00D0D0D0E03268
:100D27007594FF752F05E4F530F53190000CF0A3AD
:100D3700F090010BE054F7F054EFF054DFF054BF9C
:100D4700F0547FF090010AE054F7F054EFF054DFCD
:100D5700F054BFF0547FF0A3E054FEF054FDF0547C
:030D6700FBF0227C
:0411B300752F092269
:100DAA00E4FFEF25E025E0246CF582E43400F583C6
:100DBA00E4F0A3F00FBF20EAE4FF7F4090002CE4A8
:100DCA00F0A3DFFCE4FF741E2FF8E4F60FBF04F66D
:0D0DDA00E4FF74192FF8E4F60FBF04F622B1
:0E10AC00758911D2B4D2B9D2A9D28CD2AF229A
:100DE700AFA0EFC3135455FEEF25E054AA4EFF13EF
:100DF700135433FEEF25E025E054CC4EFF54F0FEAC
:100E0700E590540F4EF4F522EF540FF4540FF523E9
:0D0E1700120E24EFF4F52485288002082D2A
:100BCA00E4FF74222FF8E6FE743F2FF8A6060FBF43
:100BDA0006F0E4FF74282FF8E6FE74452FF8A606FF
:100BEA000FBF06F0E4FF74692FF8E6FE74202FF5B4
:100BFA0082E43401F583EEF00FBF20EAE4FF74ECDF
:100C0A002FF582E43400F583E0FE74402FF582E488
:100C1A003401F583EEF00FBF20E4E4FF741E2FF8D1
:100C2A00E6FE74362FF8A6060FBF04F0E4FF741927
:0F0C3A002FF8E6FE74322FF8A6060FBF04F02243
:100E8300756701120D27120DAA1210AC120DE7128D
:100E9300000E120647120D6A120BCAE56760EDE4F5
:070EA300F5671211B380E5B1
:10000E00E52F5401FF120F7CE51130E01CAF12EF0B
:10001E00C31320E021EF4402F512E4900070F0A328
:10002E00F0A3F0A3740AF0800DE51254FDF512E46E
:10003E00900070F0A3F0AF1EEFC3120F78121101F3
:10004E00EF5401FFE52854FE4FF5285401FF120F1F
:10005E007CE51130E01EAF12EF1313543F20E02168
:10006E00EF4404F512E4900074F0A3F0A3F0A3742F
:10007E000AF0800DE51254FBF512E4900074F0A323
:10008E00F0AF1EEF120F77121101EF5401FF25E0B2
:10009E00FFE52854FD4FF528FFC3120F78E5113008
:1000AE00E01FAF12EF131313541F20E021EF44088B
:1000BE00F512E4900078F0A3F0A3F0A3740AF08098
:1000CE000DE51254F7F512E4900078F0A3F0AF1E90
:1000DE00EF120F76121101EF5401FF25E025E0FF1C
:1000EE00E52854FB4FF528FF120F77E51130E01D80
:1000FE00AF12EFC4540F20E021EF4410F512E4903C
:10010E00007CF0A3F0A3F0A3740AF0800DE5125466
:10011E00EFF512E490007CF0A3F0AF1EEFC41210C6
:10012E00FBEF5401FF33333354F8FFE52854F74FF8
:10013E00F528FF120F76E51130E01EAF12EFC41353
:10014E00540720E021EF4420F512E4900080F0A344
:10015E00F0A3F0A3740AF0800DE51254DFF512E45B
:10016E00900080F0A3F0AF1EEFC4120F78121101B1
:10017E00EF5401FFC454F0FFE52854EF4FF528FF6C
:10018E00C45401FF120F7CE51130E01FAF12EFC413
:10019E001313540320E021EF4440F512E490008441
:1001AE00F0A3F0A3F0A3740AF0800DE51254BFF58E
:1001BE0012E4900084F0A3F0AF1EEFC4120F77127A
:1001CE001101EF5401FFC43354E0FFE52854DF4F13
:1001DE00F528FFC4120F78E51130E020AF12EFC4FE
:1001EE00131313540120E021EF4480F512E4900024
:1001FE0088F0A3F0A3F0A3740AF0800DE512547FEB
:10020E00F512E4900088F0A3F0AF1EEF120F7512F6
:10021E001101EF5401FFC4333354C0FFE52854BF1E
:10022E004FF528FFC4120F77E51130E018E51320C3
:10023E00E0204401F513E490008CF0A3F0A3F0A3AA
:10024E00740AF0800DE51354FEF513E490008CF063
:10025E00A3F0E51F1210FBEF5401FFC433333354E8
:10026E0080FFE528547F4FF528FF120F75E51130FA
:10027E00E018E51220E0204401F512E490006CF045
:10028E00A3F0A3F0A3740AF0800DE51254FEF5124C
:10029E00E490006CF0A3F0E51E5401FF120F7CE514
:1002AE001130E058E4900070F0A3F0C37470946CB9
:1002BE00FF74009400FE7C007D02120A207C007DFB
:1002CE0008120A20741E2FF8C000E6FFC007C37480
:0802DE0070946CFF74009400A1
:1002E600FE7C007D02120A207C007D08120A20AFE7
:1002F600057401A807088002C333D8FCF4FED0E0D9
:100306005ED000F6E51130E058E4900074F0A3F0FA
:10031600C37474946CFF74009400FE7C007D02121A
:100326000A207C007D08120A20741E2FF8C000E601
:10033600FFC007C37474946CFF74009400FE7C00C5
:100346007D02120A207C007D08120A20AF05740186
:10035600A807088002C333D8FCF4FED0E05ED000C4
:10036600F6E51130E058E4900078F0A3F0C3747815
:10037600946CFF74009400FE7C007D02120A207CBF
:10038600007D08120A20741E2FF8C000E6FFC00781
:10039600C37478946CFF74009400FE7C007D021296
:1003A6000A207C007D08120A20AF057401A8070800
:1003B6008002C333D8FCF4FED0E05ED000F6E5112F
:1003C60030E058E490007CF0A3F0C3747C946CFF9A
:1003D60074009400FE7C007D02120A207C007D08D9
:1003E600120A20741E2FF8C000E6FFC007C3747CF3
:1003F600946CFF74009400FE7C007D02120A207C3F
:10040600007D08120A20AF057401A807088002C300
:1004160033D8FCF4FED0E05ED000F6E51130E058AB
:10042600E4900080F0A3F0C37480946CFF74009491
:1004360000FE7C007D02120A207C007D08120A2044
:10044600741E2FF8C000E6FFC007C37480946CFFCB
:1004560074009400FE7C007D02120A207C007D0858
:10046600120A20AF057401A807088002C333D8FC1E
:10047600F4FED0E05ED000F6E51130E058E49000DE
:1004860084F0A3F0C37484946CFF74009400FE7C23
:10049600007D02120A207C007D08120A20741E2F9D
:1004A600F8C000E6FFC007C37484946CFF74009420
:1004B60000FE7C007D02120A207C007D08120A20C4
:1004C600AF057401A807088002C333D8FCF4FED038
:1004D600E05ED000F6E51130E058E4900088F0A325
:1004E600F0C37488946CFF74009400FE7C007D0257
:1004F600120A207C007D08120A20741E2FF8C00004
:10050600E6FFC007C37488946CFF74009400FE7CF9
:10051600007D02120A207C007D08120A20AF0574B5
:1005260001A807088002C333D8FCF4FED0E05ED0F1
:1005360000F6E51130E058E490008CF0A3F0C374A7
:100546008C946CFF74009400FE7C007D02120A20DD
:100556007C007D08120A20741E2FF8C000E6FFC03A
:1005660007C3748C946CFF74009400FE7C007D02BB
:10057600120A207C007D08120A20AF057401A80724
:10058600088002C333D8FCF4FED0E05ED000F6E566
:100596001130E058E4900090F0A3F0C37490946C8E
:1005A600FF74009400FE7C007D02120A207C007D10
:1005B60008120A20741E2FF8C000E6FFC007C37495
:1005C60090946CFF74009400FE7C007D02120A2059
:1005D6007C007D08120A20AF057401A80708800276
:1005E600C333D8FCF4FED0E05ED000F6E51130E06F
:1005F6004EE490006CF0A3F0FFFEFC7D02120A2090
:070606007C007D08120A20B0
:10060D00741E2FF8C000E6FFC007C3746C946CFF16
:10061D0074009400FE7C007D02120A207C007D088F
:10062D00120A20AF057401A807088002C333D8FC55
:0A063D00F4FED0E05ED000F60022CB
:03000000021137B3
:0C113700787FE4F6D8FD758188020E83F5
:100A0E00EF8DF0A4A8F0CF8CF0A428CE8DF0A42EFC
:020A1E00FE22B6
:100A2000C2D5EC30E709B2D5E4C39DFDE49CFCEEF1
:100A300030E715B2D5E4C39FFFE49EFE120AEEC371
:100A4000E49DFDE49CFC8003120AEE30D507C3E46C
:060A50009FFFE49EFE2260
:100A5600C5F0F8A3E028F0C5F0F8E582158270022B
:060A66001583E038F022C8
:100A6C00BB010A89828A83E0F5F0A3E02250068755
:100A7C00F009E71922BBFE07E3F5F009E319228917
:0B0A8C00828A83E493F5F0740193224A
:100A9700BB010789828A83020A56500B09C5F027D2
:100AA700F7C5F01937F722BBFE0D09F8E325F0F378
:100AB700C5F019E338F322F889828A8374019325F4
:080AC700F0C5F0F8E4933822B9
:100ACF00BB010A89828A83F0E5F0A3F0225006F772
:0F0ADF0009A7F01922BBFE06F3E5F009F319226F
:100AEE00BC000BBE0029EF8DF084FFADF022E4CCEC
:100AFE00F875F008EF2FFFEE33FEEC33FCEE9DECB5
:100B0E00984005FCEE9DFE0FD5F0E9E4CEFD22EDFA
:100B1E00F8F5F0EE8420D21CFEADF075F008EF2F44
:100B2E00FFED33FD4007985006D5F0F222C398FD35
:050B3E000FD5F0EA22D2
:00000001FF
